S01800006275696C642F6D696361322F6D61696E2E737265632D
S11300000C94B5010C94D2010C94D2010C94D2013D
S11300100C94D2010C94D2010C94D2010C94D20110
S11300200C94D2010C94D2010C94D2010C94D20100
S11300300C94D2010C94D2010C94D2010C94A01310
S11300400C94D2010C948B020C94B4020C94D20143
S11300500C94DE020C9474100C94D2010C94D20112
S11300600C94D2010C94D2010C944A250C94D20124
S11300700C94D2010C94D2010C94D2010C94D201B0
S11300800C94D2010C94D2010C94D20100060030DD
S1130090003C0090010F01F803D9079B0F060000F4
S11300A0000A00190032006400C8019003200640D1
S11300B03158000057F685035544020F60E0261CB2
S11300C06B55700100000000000000000081013148
S11300D07C00007BF9AE02388C3280401026A16B84
S11300E0551001000000000000000000F301315130
S11300F0000050F74F030E44020F58E026A16B5541
S113010070010000000000000000008101315CE08B
S1130110005CDB4201AA8C3280301026A16B5510A2
S113012001000000000000000000F3013145600000
S11301304555BB039C80020F68E026A16B547001F7
S11301400000000000000000008101315800005749
S1130150F685035590020F60E026A16B55700100EF
S11301600000000000000000810100002110422076
S113017063308440A550C660E770088129914AA184
S11301806BB18CC1ADD1CEE1EFF1311210027332FB
S11301905222B5529442F772D662399318837BB3D4
S11301A05AA3BDD39CC3FFF3DEE36224433420048B
S11301B00114E664C774A44485546AA54BB5288524
S11301C00995EEE5CFF5ACC58DD5533672261116DB
S11301D03006D776F6669556B4465BB77AA7199774
S11301E03887DFF7FEE79DD7BCC7C448E558866863
S11301F0A7784008611802282338CCC9EDD98EE9C4
S1130200AFF9488969990AA92BB9F55AD44AB77A3A
S1130210966A711A500A333A122AFDDBDCCBBFFB13
S11302209EEB799B588B3BBB1AABA66C877CE44C4A
S1130230C55C222C033C600C411CAEED8FFDECCD63
S1130240CDDD2AAD0BBD688D499D977EB66ED55E1A
S1130250F44E133E322E511E700E9FFFBEEFDDDFB3
S1130260FCCF1BBF3AAF599F788F8891A981CAB13F
S1130270EBA10CD12DC14EF16FE18010A100C23071
S1130280E3200450254046706760B9839893FBA32C
S1130290DAB33DC31CD37FE35EF3B1029012F322C1
S11302A0D2323542145277625672EAB5CBA5A8957C
S11302B089856EF54FE52CD50DC5E234C324A01411
S11302C081046674476424540544DBA7FAB799870C
S11302D0B8975FE77EF71DC73CD7D326F236910661
S11302E0B01657667676154634564CD96DC90EF954
S11302F02FE9C899E9898AB9ABA9445865480678B1
S11303002768C018E1088238A3287DCB5CDB3FEB6B
S11303101EFBF98BD89BBBAB9ABB754A545A376A00
S1130320167AF10AD01AB32A923A2EFD0FED6CDD3B
S11303304DCDAABD8BADE89DC98D267C076C645C50
S1130340454CA23C832CE01CC10C1FEF3EFF5DCF4B
S11303507CDF9BAFBABFD98FF89F176E367E554EA0
S1130360745E932EB23ED10EF01E11241FBECFEF49
S1130370D0E1DEBFCDBF11E0A0E0B1E0E2E3F3E6FF
S113038000E00BBF02C007900D92A235B107D9F768
S11303901EE0A2E5B1E001C01D92A23AB107E1F767
S11303A00C9422030C940000EBE5FBE081EE93E057
S11303B09F01225E3F4F819391938C5A9F4F2E173A
S11303C03F07CCF71092530B1092F50A0895FF9251
S11303D00F931F93CF93DF938C01F62EEC01809142
S11303E0F50A992701969C01807F9170281B390B8F
S11303F08091530B992728173907F9F0C8010E94F7
S1130400B70C8130D1F4888199814C819801BC0169
S11304108F2D0E94780D813081F48091F50AE82FA8
S1130420FF27EE0FFF1FE55AF44FC081D1810083EF
S113043011838F5F8F708093F50ACE01DF91CF9186
S11304401F910F91FF900895AF92BF92CF92DF92C8
S1130450EF92FF920F931F93CF93DF9306EEA0903A
S11304608D0EB0908E0EC0908F0ED090900EA11471
S1130470B104C104D104C9F110E06DE77BE0EE24BE
S1130480FF2481E090E0A0E0B0E00E2C04C0880FCF
S1130490991FAA1FBB1F0A94D2F78A219B21AC2162
S11304A0BD210097A105B10579F0202F33274427FA
S11304B05527FB0185819681A781B0858217930713
S11304C0A407B5070CF405811F5F0894E11CF11C17
S11304D0675F7F4F1A30A8F28FB7F894992712B745
S11304E01D5F011728F4012F03C08FB7F8949927D3
S11304F00093490D01BF1092270D8FBF0E94D708AA
S1130500DF91CF911F910F91FF90EF90DF90CF90EB
S1130510BF90AF9008951F920F920FB60F921124BF
S11305202F933F934F935F936F937F938F939F93F7
S1130530AF93BF93EF93FF939FB18091BC0A8FB9A0
S1130540892F0E94E61EFF91EF91BF91AF919F9179
S11305508F917F916F915F914F913F912F910F9068
S11305600FBE0F901F9018951F920F920FB60F9207
S113057011242F933F934F935F936F937F938F93A4
S11305809F93AF93BF93EF93FF935F9B06C08CB190
S113059040E050E060E00E949626FF91EF91BF9109
S11305A0AF919F918F917F916F915F914F913F9107
S11305B02F910F900FBE0F901F90189578941F9253
S11305C00F920FB60F9211242F933F934F935F9383
S11305D06F937F938F939F93AF93BF93EF93FF9307
S11305E00E946228FF91EF91BF91AF919F918F91EB
S11305F07F916F915F914F913F912F910F900FBE1B
S11306000F901F901895BC018FB7F894482F552769
S113061020911F0DE22FFF27EE0FFF1FE75BF54F21
S113062080819181892B51F42F5F277020931F0DB6
S1130630608371834FBF81E090E008954FBF80E0F5
S113064090E00895CDEFD0E1DEBFCDBFD698A79A54
S1130650A69AA59AA49AA39AA29AA19AA09A8C9AC5
S11306608F9A8E9ABB98BF98D498DC9883E08C5F5D
S11306708739E8F390E08AE08093720290931F0D2B
S11306809093F00A89E49AE0FC019C01225F3F4FB9
S113069011921192029628173907D4F70E94140771
S11306A00E94D4010E9414070E9443078FB7F89454
S11306B099271092330D8FBF8FB7F894682F77273F
S11306C082E080936802809354018CEF9AE09093C7
S11306D0250D8093240D1092000B8BE490E09093F1
S11306E0100D80930F0D1092E00310920E0D1092D6
S11306F0960E1092950E1092DD031092DC03109268
S11307005B0A10925A0A10929A0E10921A021092D0
S11307100B0210925E0D10920D0D41E040935F0AA2
S11307208CE291E090933B0D80933A0D2FEF3FEFD5
S11307303093350D2093340D3093370D2093360DBF
S113074010925C0A10920D021092460D10926D02E6
S113075080E291E09093510B8093500B10920C0225
S113076010925D0D10925C0D1092F40A1092F30A2F
S11307701092160D1092150D80E090E0A0E0B0E00C
S11307808093620290936302A0936402B093650223
S11307901092570B1092580B1092590B10925A0B3F
S11307A080E290E09093DB038093DA0390937602E7
S11307B08093750282E390E090932E0E80932D0E29
S11307C080E496E09093560B8093550B90932C0EF7
S11307D080932B0E1092C10D1092310E1092520B79
S11307E010921E0D1092620A4093780310927703C0
S11307F01092240E1092230E10925601109255015D
S11308001092120D1092110D4EED4093BA0C3093CC
S1130810B90C2093B80C85E08093BC0C9DE79093B1
S1130820BB0C1092040D1092030D40936D0D309388
S11308306C0D20936B0D80936F0D90936E0D109241
S1130840B70D1092B60D8FED8093670A3093660A48
S11308502093650A87E08093690A9093680A10924E
S1130860B10A1092B00A1092BD0C80912F0D909194
S1130870300D9093BF0C8093BE0C80910001909139
S113088001019093C10C8093C00C6FBF28E0ECE190
S1130890F2E080E291E081939193215027FFF9CF18
S11308A08FB7F8949927B998BB98BA986B986A98B7
S11308B06F9A6E9A8FBF81E480938A00D6988C9A3F
S11308C08E9A8F9A949A979A969A6AE380E00E94F5
S11308D087076BE380E00E94870780ED97E00000C4
S11308E0000000000000000000000000000001976C
S11308F018161906A4F380E88093DA0A682F8BE0AF
S11309000E94870780E98093DC0A682F84E00E94B4
S113091087071092DE0A8FE68093DF0A85E58093CD
S1130920E00A6091DE0A8FE00E9487078091DF0A67
S1130930682F80E10E9487078091E00A682F81E197
S11309400E94870711E01093E20A612F83E10E945D
S113095087071093ED0A8FEC9AE0DC011196E1EB26
S1130960F0E09C01225E3F4F84918D9331962A17CB
S11309703B07D4F711E050EDE52E5AE0F52EF701D0
S113098081917F01682F812F0E9487071F5F1D308F
S1130990B0F38091E10A682F82E10E94870760E04A
S11309A08BE00E9487076FE382E40E94870761E17E
S11309B080E00E94870766EA8EE00E9487078EE047
S11309C00E94AB0783FFFBCF66E28EE00E9487079D
S11309D061EE80E00E9487078091EC0A682F89E02D
S11309E00E94870760E08BE00E94870766EA8EE03A
S11309F00E9487071EE0812F0E94AB0783FFFACF76
S1130A0066E2812F0E94870780E98093DC0A682FC1
S1130A108DE00E9487078091ED0A8093260E0E9444
S1130A20DE078FB7F89499271092C20D8FBF8FB746
S1130A30F894282F33271092F90A1092F80A10928A
S1130A40230D1092220D10929F0E10929E0E109262
S1130A507C0B10927B0B8DE791E0A0E0B0E08093DB
S1130A60910E9093920EA093930EB093940E2FBF79
S1130A700E94DE078FB7F894992716B917B88FBF6D
S1130A800E94F9070E9414078091000190910101CE
S1130A909093370E8093360E10924A0D109267028F
S1130AA0109266021092460A1092450A1092B70CF0
S1130AB081E080931B0280E090E00EC0FC0143E0E3
S1130AC0EE0FFF1F4A95E1F7E81BF90BE952F44FCB
S1130AD01282158216820196803291057CF310925F
S1130AE00C0D10925301109252011092980E109214
S1130AF0970E81E080932A0EE1E2F9E08FE191E024
S1130B00119201972FEF8F3F9207D1F78EE790E074
S1130B109093BE0A8093BD0A9093C00A8093BF0A43
S1130B2021E02093CA0A1092CC0A10926A02109211
S1130B3069028FEF8093260D1092420A1092410AA7
S1130B401092440A1092430A80E090E2A0E0B0E0E0
S1130B5080936E0290936F02A0937002B09371021F
S1130B6010923C0D209360020E9414071092210DF4
S1130B701092200D1092390D1092380D1092300EF3
S1130B8010922F0E0E94290880E0EEE2F2E011920A
S1130B908F5F8233E0F3109279031092350E109236
S1130BA090008FE089B982E08BB986E0809395004C
S1130BB08CB188E08AB981E080937B031092D903D9
S1130BC00E94F9070E944307109290008FE089B9B0
S1130BD082E08BB986E08093950088ED8AB98FB75F
S1130BE0F8949927409168028FBF6FEF7FEFA3E0DD
S1130BF08FB7F894282F332780917D008F7E8093C0
S1130C007D008BE080938A00109289001092880006
S1130C10709387006093860010928B0080918B0004
S1130C20806480938B00139A10928C0080917D00D5
S1130C30806180937D002FBF10927A03423009F0C7
S1130C407DC08FB7F894482F5527E091240DF0917B
S1130C50250D1482A093680210920B0210921A02BE
S1130C607093350D6093340D1092540B1092460D11
S1130C70EEE9F0E084919927382F22273196849168
S1130C809927282B392B3093320D2093310DECE822
S1130C90F0E084919927382F22273196849199275F
S1130CA0282B392B3093D2032093D1034FBFE091EB
S1130CB0240DF091250D14828FB7F8949927A093F1
S1130CC068028FBF6BE380E00E94870769E380E0DE
S1130CD00E94870788EC90E00000000000000000FC
S1130CE00000000000000000019718161906A4F384
S1130CF0BB98BA980E94480880910E0D8F3128F055
S1130D0020E03AE040E050E004C020E830E040E079
S1130D1050E060E084E00E94670880EC8DB9B898E8
S1130D200E94D7088091460D882341F020E03AE0E4
S1130D3040E050E061E085E00E94670828EE33E07F
S1130D4040E050E060E083E00E9467080E94D7081A
S1130D5010924A0D209100013091010121153105B5
S1130D6061F48DEB9AE090936A0280936902109289
S1130D70260D3093180D2093170D8091600288235F
S1130D8091F089EE98E00E94030380916E029091A5
S1130D906F02A0917002B09171029C01AD0160E0FC
S1130DA088E00E94670811E01093B70CAE014F5F12
S1130DB05F4F6FEC7DE08DE40E94780AFC01809126
S1130DC0000180838FEF8093DA0A0E94800A60E634
S1130DD07AEE0E946331AA27BB279C01AD01612FE3
S1130DE080E00E94670878948FB7F894482F5527BD
S1130DF09091F00AE92FFF27EE0FFF1FE75BF54FF5
S1130E00208131812115310529F4789488950000D9
S1130E100000EACF108211829F5F97709093F00ACE
S1130E204FBFF9010995E0CF10928D0E10928E0EEE
S1130E3010928F0E1092900E1092270D8FEF8093C8
S1130E40990E809303021092470A83E080932A0D3F
S1130E5096EE9093490D8FB7F894282F332787B7D0
S1130E608E7F87BF87B78D7F87BF80B7886080BF3D
S1130E708BE083BF12BE91BF87B7826087BF2FBF4D
S1130E8081E090E008958FB7F894682F80E090E0B7
S1130E9049E551E09C01F901E80FF91FE55BF24FC8
S1130EA04483558312821382118201962B5F3F4F34
S1130EB04C5A5F4F8230910574F31092250E1092B4
S1130EC0140D1092130D10926C0210926B0210927A
S1130ED058011092570110920202109201021092CE
S1130EE0CE0D10923D0D1092270E10927E0310929B
S1130EF07D031092610A1092600A80914F0D9091C7
S1130F00500D9093650D8093640D6FBF0895880F05
S1130F10949896E087FF02C0979A01C09798969894
S1130F20969A880F915097FFF5CF979A9698969A2C
S1130F30949A97E067FF02C0979A01C09798969891
S1130F40969A660F915097FFF5CF949A979A969A2E
S1130F5081E090E0089590E0880F949826E030E0D6
S1130F6087FF02C0979A01C097989698969A880F1F
S1130F702150304037FFF4CF27E030E0979896981F
S1130F80969A8F98949A969840E050E0879941E019
S1130F90892F992721503040442329F0880F991F25
S1130FA0982F916002C0982F990F969A37FFEBCF34
S1130FB0949A8F9A979A892F992708958FB7F894BE
S1130FC0282F80917C03882391F480E090E0E2EC68
S1130FD0FDE0819301968C309105DCF38EE18093E2
S1130FE0CC0D8FE18093CD0D81E080937C032FBFE6
S1130FF008958FB7F894482F552720910001309118
S1131000010181E597E3289FB001299F700D389F66
S1131010700D1124CB018F5A984C90935A0D8093E4
S1131020590D90939C0E80939B0E85E89FE0289F1A
S1131030B001299F700D389F700D1124CB018B577F
S1131040904F90937402809373024FBF81E090E0BD
S113105008951092580D1092570D10921D0D109274
S11310601C0D1092D0031092CF031092340E1092E4
S1131070330E109205021092040210922C0D10925D
S11310802B0D1092F70A1092F60A81E090E0089571
S11310908091D80A682F89E00E94870760E08BE07E
S11310A00E94870761E180E00E9487078DE790E056
S11310B0000000000000000000000000000000002C
S11310C0019718161906A4F381E090E00895EF92B1
S11310D0FF920F931F93CF93DF93962F79018A0189
S11310E08A3050F4623044F4662349F423E0E21673
S11310F0F1040105110518F480E090E051C0682F57
S11311007727FB01A3E0EE0FFF1FAA95E1F7E60F97
S1131110F71FE358F44FE182F28203831483908330
S11311208FB7F894C82FDD2782B7E80EF11C011D94
S1131130111DE582F6820783108721E030E040E04C
S113114050E004C0220F331F441F551F6A95D2F785
S113115080918D0E90918E0EA0918F0EB091900E75
S1131160822B932BA42BB52B80938D0E90938E0EF4
S1131170A0938F0EB093900E8091490D9927AA27C2
S1131180BB27E816F9060A071B0738F4E092490D55
S1131190E1BE1092270D0E94D708CFBF81E090E0F6
S11311A0DF91CF911F910F91FF90EF90089580915F
S11311B0080118162CF082ED9AE20E94030306C07F
S11311C085B7837E85BF85B7806285BF80E090E068
S11311D008952F923F924F925F926F927F928F92D7
S11311E09F92AF92BF92CF92DF92EF92FF920F93B2
S11311F01F93CF93DF93CDB7DEB723970FB6F89441
S1131200DEBF0FBECDBF10E08091430A9091440A27
S113121001966AE070E00E9463319093440A8093DF
S1131220430A6C01E1E2F9E08585992780FF4DC00E
S1131230C114D10409F049C032E0A32EB12CA82274
S1131240B92281FD42C08FB7F894482F2185328599
S113125067817085620F731F6A30710510F46AE04C
S113126070E08FEF90E0289FD001299FB00D389F48
S1131270B00D1124CD010E946331A782B086A186EE
S1131280B2868685882321F481898695818B02C064
S1131290815086874FBF958592FF0EC0CB01880F82
S11312A0991F860F971F2089820F911D9695879508
S11312B096958795808B04C0608B84E098279587EA
S11312C08681882311F0815086831F5F72961031C6
S11312D008F4AACF1FEFA12E1FEFB12E1FEFC12ECE
S11312E01FEFD12E25013601882499241401809101
S11312F0000190910101892B09F4A5C01982E1E252
S1131300F9E0EA83FB83EA81FB81858580FF4EC097
S113131022813381809100019091010128173907BE
S113132009F444C02F3F310509F440C087858F3F3D
S1131330E9F1848195818F3F9105C1F1618969311A
S1131340A8F14089493190F18681882379F580E0BC
S113135090E00E94440A7B018C01EA81FB81408970
S11313606189848195810E94440A9B01AC01F1E06A
S1131370EF16F6E0FF06F0E00F07F0E01F07B0F409
S11313808091690290916A026A817B81681779076A
S113139021F41B0129013A0109C02A153B054C051A
S11313A05D0520F459016A018A809B8079817F5F01
S11313B079838A819B8142968A839B83703108F466
S11313C0A2CF8114910471F02114310471F0D6017B
S11313D0C50180589E4FAF4FBF4F481659066A0645
S11313E07B0618F441016301520181149104C9F090
S11313F08FB7F894282F332790926A02809269025B
S1131400F40187858F5F8093260DB6E0D694C79448
S1131410B794A794BA95D1F7B092180DA092170D6E
S113142011C08FB7F894282F332790926A028092C4
S113143069028FEF8093260D8FEF90E09093180D43
S11314408093170D2FBF20E230E040E050E061E0D0
S113145089E00E94670823960FB6F894DEBF0FBE9A
S1131460CDBFDF91CF911F910F91FF90EF90DF904F
S1131470CF90BF90AF909F908F907F906F905F9030
S11314804F903F902F900895CF93DF93EC01862FD8
S1131490242F9927AA27BB27332744275527BC0184
S11314A0CD010E9438319B01AC01611571058105A4
S11314B0910529F420E030E041E050E014C060E000
S11314C070E080E091E00E947731CE01AA27BB272B
S11314D066E0880F991FAA1FBB1F6A95D1F7280FD2
S11314E0391F4A1F5B1FCA01B901DF91CF910895CB
S11314F0CB01FA012FE330E0208331830C96089569
S11315008FB7F894482F55272091590D30915A0DD3
S1131510832F881F8827881F220F331F882321F0D9
S11315208BE090E1282739272F5F3F4F30935A0DE6
S11315302093590D809173029091740228273927C2
S11315404FBFC9010895CF92DF92EF92FF920F939C
S11315501F93CF93DF93CDB7DEB721970FB6F894DF
S1131560DEBF0FBECDBF7C018091450A9091460A33
S113157001969093460A8093450AF70193818091DE
S11315800201981709F0BDC08091B70C813071F049
S113159020813181FFEF2F3F3F0741F0809100010F
S11315A0909101012817390709F0ABC080911B0203
S11315B0882371F02BE430E0E20EF31EF701808102
S11315C0918125EB3FEFE20EF31E019709F099C0DC
S11315D0F701928180E08B5E8435E8F3892F9927A7
S11315E08D34910569F08E3491051CF4039729F02C
S11315F084C08A3F910549F080C0B70183E002C0EE
S1131600B7018DE40E94690C79C087010B5F1F4FFD
S11316103CE0C32ED12CCE0CDF1CF70185819681D2
S1131620AE014F5F5F4FF801648175810E94910B99
S11316306981862F9927DC0124E0AA0FBB1F2A9514
S1131640E1F7A80FB91FA80FB91FAF5DB64FF70197
S11316508485958512968D939C931397F8018681C2
S11316601F968C931F97F6018281938114968D9314
S11316709C93159716968C911697882361F0F70121
S1131680248535858091000190910101281739073F
S113169011F016961C9220E0F6018481281768F553
S11316A04091000150910101822F9927DC01AA0F7A
S11316B0BB1FA80FB91FAC0DBD1DFD0115968D9163
S11316C09C9116978417950799F4862F99278C0176
S11316D0A4E0000F111FAA95E1F7080F191F080FC6
S11316E0191F0F5D164F8781F801818B85E086876E
S11316F02F5FF60184812817B8F2C701009709F01B
S11317007C01C70121960FB6F894DEBF0FBECDBF92
S1131710DF91CF911F910F91FF90EF90DF90CF90C9
S11317200895AF92BF92CF92DF92EF92FF920F9300
S11317301F93CF93DF938C017B015A01CC240E9429
S1131740280CC82F8F3F11F5A82FB82F9C2D40E0EF
S113175050E09A01B901FA01E20FF31FEF5DF64F71
S1131760858580FF3FC08189A81710F0A82FB92F65
S11317709F5F9B012F5F3F4F4F5E5F4F903150F350
S11317808B2F9927C82FB8010E94460CAC2FBB277A
S1131790DA2E82E1A89FE0011124CF5DD64F8A2F73
S11317A09927FC0154E0EE0FFF1F5A95E1F7E80F6B
S11317B0F91FE80FF91FEF5DF64F838594859701B4
S11317C0281B390B215030404D8541FF0DC08985C0
S11317D09A85019689879A87EB86FC8682E048275A
S11317E04D8727C0C901CECF37FD0EC08F819885A4
S11317F0820F931F8F83988789859A85019689879D
S11318009A87EB86FC8615C02C5E3F4F84F4B801A2
S11318108A2F0E94460C89859A85019689879A8722
S1131820EB86FC868D8592E089278D8702C041E096
S1131830C42EF501D0828C2D9927DF91CF911F9171
S11318400F91FF90EF90DF90CF90BF90AF900895ED
S1131850BC01A0E020E030E0A901FA01E20FF31F8F
S1131860EF5DF64F858580FF07C0808191818617E3
S1131870970711F4C9010895AF5F4F5E5F4F2F5F63
S11318803F4FA03150F38FEF90E008959B019927CB
S1131890FC0164E0EE0FFF1F6A95E1F7E80FF91F02
S11318A0E80FF91FEF5DF64F2083318383E08587CE
S11318B016868FEF90E082839383848395831682C8
S11318C08FEF87871782108611861286108A118AF5
S11318D008950F931F93CF93DF93CDB7DEB721976E
S11318E00FB6F894DEBF0FBECDBF482F8B01FB01AE
S11318F03596DB012D913C911197809100019091D7
S1131900010128173907E1F44D34A1F41C968C9198
S1131910823380F4E82FFF27E25DFD4F80818F5FE3
S113192080838091200D9091210D01969093210D3B
S11319308093200D642FC8010E94E7018C010BC025
S1131940AE014F5F5F4F6481758115968D919C91B7
S113195016970E94910BC80121960FB6F894DEBF2A
S11319600FBECDBFDF91CF911F910F910895DF92EC
S1131970EF92FF920F931F93CF93DF93CDB7DEB710
S113198021970FB6F894DEBF0FBECDBF7C018C014A
S11319900B5F1F4FE1E0DE2E8091690290916A0295
S11319A0892B51F5F70125813681809100019091B1
S11319B001012817390731F5F801828193818217D3
S11319C0930701F5F701858396838091260DF8012D
S11319D086838091410A9091420A8483958301967B
S11319E09093420A8093410A8FEF9FEFF70180831F
S11319F0918381E090E06EC09091260DF80186817C
S1131A00981718F080E090E065C0F70125813681D1
S1131A1080910001909101012817390741F4F801E0
S1131A20828193818217930711F480E00AC0AE018A
S1131A304F5F5F4FF80164817581808191810E94BD
S1131A40910B882309F043C080910001909101011A
S1131A50F801808391838091260D8683A091690289
S1131A60B0916A028D919C9111978E37910559F02E
S1131A708091410A9091420A8483958301969093C0
S1131A80420A8093410A8D919C91F701808391834E
S1131A90F80122813381809100019091010128177E
S1131AA03907B1F0C9010E94280C8F3F89F09927AA
S1131AB0FC0174E0EE0FFF1F7A95E1F7E80FF91FC0
S1131AC0E80FF91FEF5DF64F85E0868301C0DD2442
S1131AD08D2D992721960FB6F894DEBF0FBECDBF8A
S1131AE0DF91CF911F910F91FF90EF90DF900895B8
S1131AF0CF93DF93582FE901A0915201B091530184
S1131B00CD0101968F7190702091970E3091980EAF
S1131B108217930711F0473418F020E030E02FC00B
S1131B20209711F49E012BC0FD0183E0EE0FFF1FEF
S1131B308A95E1F7EA1BFB0BE952F44F608371834A
S1131B4042835383C583D6831482C15BDF4F1882DB
S1131B50809152019091530101968F7190709093EE
S1131B6053018093520180912A0E882331F0109200
S1131B702A0E83EC9DE00E94030321E030E0C901BA
S1131B80DF91CF910895DF92EF92FF920F931F930D
S1131B90CF93DF938091970E9091980EFC0123E0F0
S1131BA0EE0FFF1F2A95E1F7E81BF90BE952F44FFA
S1131BB0C581D6812097A9F1D380E080F18002818C
S1131BC010914A0D112321F581E080934A0D0734C9
S1131BD030F482E399E20E940303882319F41093FA
S1131BE04A0D16C0D0933F0DC0933E0D0C83E8827E
S1131BF0F982DA82E0913E0DF0913F0D809102016D
S1131C008383812F8B5E8435E8F381E090E002C00A
S1131C1080E090E0892B41F483EC9DE00E94030373
S1131C2003C081E080932A0EDF91CF911F910F9121
S1131C30FF90EF90DF900895CF93C1E020E08FB73D
S1131C40F894382F8091250E8823C9F580919D0E34
S1131C50992781FF09C080E49DE09093EF0A809367
S1131C60EE0A80E490E01EC082FF12C0E0910102FF
S1131C70F0910202F093EF0AE093EE0A82E490E01E
S1131C8090930A028093090284819927059610C0D3
S1131C9083FF15C081E692E09093EF0A8093EE0AE9
S1131CA08FEF90E090930A028093090281E090E024
S1131CB090936C0280936B022C2FC093250E3FBF30
S1131CC02223F1F08FB7F8949927109258011092BB
S1131CD057011092140D1092130D8FBF8EE70E94BE
S1131CE0840EC82F813061F08FB7F894282F3327E2
S1131CF088E08093250E2FBF8DE99EE00E940303A8
S1131D008C2F9927CF910895482F8FB7F894282FB7
S1131D1033279091330D81E08093330D2FBF9923A6
S1131D2019F080E090E008958FB7F89499274CB9A2
S1131D305E9A8FBF81E090E0089561E08FB7F894D8
S1131D40282F33278091250E883019F460E06093A2
S1131D50250E2FBF8091090290910A0240919D0E99
S1131D608034910551F48FB7F894282F332782E0FB
S1131D70482740939D0E2FBF17C08FB7F894282F84
S1131D80332784E0482740939D0E2FBF80910102A2
S1131D90909102020E94D70E8FB7F894992710925F
S1131DA00202109201028FBF0E941C0E08951F931D
S1131DB0CF93DC01462F10924A0D12961C91129774
S1131DC08091970E9091980EFC0153E0EE0FFF1F47
S1131DD05A95E1F7E81BF90BE952F44F8581968196
S1131DE0A817B90709F042C080910C0D882361F04F
S1131DF0A15BBF4FCC91AF54B040CC2329F4808178
S1131E0091818E37910549F4BD01812F0E943B0FCA
S1131E101A3F89F410923C0D0EC084818F5F848335
S1131E20863000F14C2FBD01812F0E943B0F1A3FD9
S1131E3011F4C0933C0D8091970E9091980EFC0183
S1131E4033E0EE0FFF1F3A95E1F7E81BF90BE95277
S1131E50F44F1582168201968F7190709093980EAC
S1131E608093970E83EC9DE00E94030381E090E051
S1131E70CF911F910895A82F5091530BE52FFF2761
S1131E80EE0FFF1FE55AF44F20813181621773076B
S1131E9029F45F5F5F705093530B15C08A2F992705
S1131EA08330910581F08D34910569F4413049F412
S1131EB08091380D9091390D01969093390D80934E
S1131EC0380D1092350E81E090E008951F93CF9362
S1131ED0FC0111E090E08FB7F894C82F80910B02B9
S1131EE0882311F0192F2BC010930B02F093C00D0F
S1131EF0E093BF0D8481992705969093DF03809327
S1131F00DE0380915F0A882399F080910C02882374
S1131F1031F40E94800A8F719070019604C080E0B1
S1131F2090E00E94F00F9093350D8093340D04C01F
S1131F301092350D1092340D81E080931A02909125
S1131F406802CFBF112309F446C0983009F043C09A
S1131F508FB7F894282F332783E0809368022FBF2C
S1131F6085E00E942C106BE380E00E94870769E300
S1131F7080E00E94870788EC90E0000000000000E9
S1131F800000000000000000000001971816190668
S1131F90A4F30E944808BB98BA9880EC8DB9B8980D
S1131FA00E94D70880910E0D8F3128F020E03AE08E
S1131FB040E050E004C020E830E040E050E060E061
S1131FC084E00E94670820E230E040E050E061E0F5
S1131FD085E00E946708812F9927CF911F9108956A
S1131FE09C0160912D0D70912E0D4091280D509102
S1131FF0290D892B11F180915C0D90915D0D019655
S113200090935D0D80935C0D6417750719F4283067
S11320103105B0F46417750771F02830310558F4B0
S1132020C901089688329105B0F00E94800A8F7128
S1132030907009960895C90108956417750731F4DD
S11320400E94800A87709070019608950E94800A09
S11320508F71907009960895CF93DF938A3008F0BA
S11320603EC041E050E060E070E004C0440F551F02
S1132070661F771F8A95D2F7C0918D0ED0918E0E70
S1132080E0918F0EF091900ECE01DF018423952311
S1132090A623B7230097A105B10509F18FB7F894DA
S11320A0282F3327DB01CA0180959095A095B09520
S11320B08C239D23AE23BF2380938D0E90938E0E8D
S11320C0A0938F0EB093900E2FBF0097A105B1057A
S11320D019F481E08093270D81E090E002C080E054
S11320E090E0DF91CF9108951F920F920FB60F9257
S11320F01124CF92DF92EF92FF920F931F932F93AD
S11321003F934F935F936F937F938F939F93AF937B
S1132110BF93CF93DF93EF93FF93C4B1D5B1D37043
S1132120349A37987894EFEF00E011E08091F80A40
S11321309091F90A0A9759F4CE01AA27BB278093F4
S1132140910E9093920EA093930EB093940E8FB72A
S1132150F894F82FD090F80AED2CFF2461E070E099
S11321600E2C02C0660F771F0A94E2F740919E0E70
S113217050919F0E462357234115510551F48091E8
S11321807B0B90917C0B8627972790937C0B8093F5
S11321907B0B2091220D3091230DCB0182239323BD
S11321A0892B49F0012F452B31F42627372730930B
S11321B0230D2093220D40917B0B50917C0B4115F4
S11321C0510501F12091F80A3091F90A2F5F3F4F30
S11321D02C30310511F0C90102C080E090E09C016F
S11321E081E090E0022E02C0880F991F0A94E2F762
S11321F084239523892B51F33093F90A2093F80A09
S1132200E091F80AFFBFEF3F19F08E2F0E9462128F
S11322108AE0D81609F421C1002311F010E01DC191
S1132220E114F10409F017C18FB7F894C82E209176
S11322306802822F99278430910529F18530910510
S11322401CF4039741F004C18630910591F009977D
S113225009F47CC0FDC080916D02833009F04CC04C
S1132260D093BB0AC093BA0A84E792E10E940303A5
S113227043C080916D02863009F03EC0D093370D83
S1132280C093360D39C080919A0E8F5F80939A0E59
S11322908091500B9091510B40968C179D0720F024
S11322A080915F0A882359F580916D02843039F555
S11322B01AEA8FB7F89499271093BC0A8FBF0E942B
S11322C01D13BB9ABA9AD093370DC093360D85E08F
S11322D080939A0E81E080935E0DF092290EE09235
S11322E0280EF092640AE092630A8093680282E006
S11322F0809354011093660D00936D02A9C010924F
S11323006D0280919A0E8530B1F480915C0D9091AC
S11323105D0D019690935D0D80935C0D0E94800A83
S11323208F70907001969093350D8093340D83E0F7
S1132330809368028DC020936D028FB7F894082FA4
S1132340112780E00E944C130FBF82C0F02E8091B1
S1132350500B9091510B9C013695279536952795F6
S1132360821B930B8C179D0748F4D093BB0AC09330
S1132370BA0A84E792E10E94030349C080910D02E6
S1132380863098F00E94480883E080936802BB98E6
S1132390BA9880EC8DB9B8980E94D7088EE793E17B
S11323A00E940303E1E0FE2E32C00E9448088FB76A
S11323B0F894082F11278F2D0E944C130FBF8823E8
S11323C0A9F080E590E0000000000000000000009B
S11323D0000000000000019718161906A4F380916C
S11323E00D028F5F80930D0271E0F72E80911C0D1A
S11323F090911D0D019690931D0D80931C0D6FE31C
S113240080E00E94870760E08BE00E94870780914C
S11324101A02882391F00E94480883E0809368029E
S1132420BB98BA9880EC8DB9B8980E94D7088EE70B
S113243093E10E94030361E0F62EFF2049F481EF4B
S113244099E20E94030388E0809368020E94981333
S1132450CFBE81E001C080E0182F8FB7F894682FB9
S113246041E050E002C0440F551FDA94E2F7209196
S11324709E0E30919F0EC90184239523892B41F030
S1132480112331F42427352730939F0E20939E0E79
S11324906FBFFF91EF91DF91CF91BF91AF919F916A
S11324A08F917F916F915F914F913F912F911F91E8
S11324B00F91FF90EF90DF90CF900F900FBE0F9091
S11324C01F901895982F8FB7F894282F3327E2EC94
S11324D0FDE0E90FF11D80818F7187B92FBF379A15
S11324E0369A81E090E008950F931F93CF93DF9382
S11324F0CDB7DEB762970FB6F894DEBF0FBECDBF7F
S11325008FB7F894482F552720915C0AE22FFF27B4
S1132510EE0FFF1FE45EFD4F8091BA0A9091BB0A53
S113252080839183822F8F5F80935C0A893010F0BF
S113253010925C0A80910E0D8F3118F48F5F809396
S11325400E0D4FBF48E0ACE1B2E020E030E0FE0108
S1132550E20FF31F8D919D918183928341502E5FF1
S11325603F4F47FFF4CF50E0A52F41E022E030E099
S1132570BE016F5F7F4FF901E60FF71F80819181E4
S1132580EFEF8F3F9E0791F0EA2FFF27E7FDF095CD
S1132590EE0FFF1FE60FF71F0190F081E02DE81703
S11325A0F90718F0EF5FFF4F09F4A42F4F5F2E5F78
S11325B03F4F4930ECF2EA2FFF27E7FDF095EE0F8D
S11325C0FF1FE60FF71F608171818FEF9FEF8083FC
S11325D091835F5F53304CF28091500B9091510B7B
S11325E0B5E0880F991FBA95E1F79C014427552758
S11325F0660F771FCB01AA27BB27280F391F4A1F55
S11326005B1F8FB7F894082F1127CA01B90122E282
S113261030E040E050E00E9477313093510B20933A
S1132620500B0FBF62960FB6F894DEBF0FBECDBF3E
S1132630DF91CF911F910F91089561EE80E00E9488
S113264087078091EC0A682F89E00E9487078AEF48
S113265090E0000000000000000000000000000006
S11326600000019718161906A4F38091DA0A682F5E
S11326708BE00E94870784E190E0000000000000E6
S11326800000000000000000000001971816190661
S1132690A4F381E090E00895CF93DF93782F41E095
S11326A050E061E0C82FDD270C2E02C0440F551FF7
S11326B00A94E2F720917B0B30917C0BCA018223B0
S11326C09323892B11F060E014C0CA01822B932B51
S11326D090937C0B80937B0B232B59F4872F0E94C0
S11326E062129927682F882321F0D093F90AC093A6
S11326F0F80A862F9927DF91CF91089580910E0DC6
S11327008F3128F020E03AE040E050E004C020E8B7
S113271030E040E050E060E084E00E9467082EE191
S113272030E040E050E061E085E00E9467080895F1
S11327306F98B89AC0980E94D70881E090E00895F5
S113274078941F920F920FB60F9211242F933F93F8
S11327504F935F936F937F938F939F93AF93BF93A5
S1132760CF93DF93EF93FF938FB7F894282F3327FA
S11327708091480A882369F08091190D8093630D34
S113278088608093190D83BF8091590A81BF10928C
S1132790480A2FBF8FB7F894C82FDD2780911A0DF0
S11327A090911B0D892B21F48EEF99E20E94030373
S11327B021B780911A0D90911B0D820F911D0196E6
S11327C090931B0D80931A0DCFBFFF91EF91DF9172
S11327D0CF91BF91AF919F918F917F916F915F91B5
S11327E04F913F912F910F900FBE0F901F9018950E
S11327F08F929F92AF92BF92CF92DF92EF92FF920D
S11328000F931F93CF93DF93CDB7DEB724970FB603
S1132810F894DEBF0FBECDBFC90120E090932E0E09
S113282080932D0E862F99279093300D80932F0D32
S1132830EFE7F3E08FEF80838183828313822F5F3E
S113284034962431B8F380910001909101018230D3
S11328509105E9F584E090E09093290D8093280D8B
S113286080E190E090937602809375028CE18093EE
S11328707F0302E00093820310E11093810383E05D
S113288080938003612F0E948B1D8BE180938303CF
S1132890009386031093850385E080938403612F5E
S11328A00E948B1D1092870300938A03109389035F
S11328B089E080938803612F0E948B1D85E18093BA
S11328C08B0300938E0310938D038DE03CC58330FE
S11328D0910509F075C08EE090E09093290D8093E6
S11328E0280D80E190E090937602809375028FE149
S11328F080937F0302E00093820310E1109381032D
S113290035E0F32EF0928003612F8F2D0E948B1DF2
S11329108FE080938303009386031093850386E0FE
S113292080938403612F0E948B1D89E28093870327
S113293000938A03109389038CE080938803612FAA
S11329400E948B1D88E280938B0300938E03109367
S11329508D038BE080938C03612F0E948B1D80E29A
S113296080938F0300939203109391030093900339
S1132970612F802F0E948B1D81E18093930300932C
S113298096031093950384E080939403612F0E942F
S11329908B1D8AE28093970300939A031093990303
S11329A087E080939803612F0E948B1D8BE18093B5
S11329B09B0300939E0310939D03F0929C0372C1AA
S11329C089309105E9F581E090E09093290D809399
S11329D0280D80E190E0909376028093750285E162
S11329E080937F0302E00093820310E1109381033C
S11329F08DE080938003612F0E948B1D8CE1809376
S1132A008303009386031093850383E080938403F8
S1132A10612F0E948B1D8BE18093870300938A03AF
S1132A201093890385E080938803612F0E948B1D96
S1132A3010928B0300938E0310938D0389E083C45B
S1132A408732910519F482E090E0BAC68A30910584
S1132A50D9F51092290D1092280D80E190E0909301
S1132A6076028093750285E180937F0302E00093F0
S1132A70820310E1109381038DE080938003612F22
S1132A800E948B1D10928303009386031093850389
S1132A9089E080938403612F0E948B1D8CE18093D5
S1132AA0870300938A031093890383E08093880348
S1132AB0612F0E948B1D8BE180938B0300938E0307
S1132AC010938D0385E03FC48831910519F487E0A4
S1132AD090E076C68130910539F586E090E09093D8
S1132AE0290D8093280D80E190E0909376028093E5
S1132AF0750285E180937F0302E00093820310E175
S1132B00109381038DE080938003612F0E948B1DBD
S1132B1085E28093830300938603109385038AE000
S1132B2080938403612FDAC68531910509F0BDC015
S1132B308DE090E09093290D8093280D80E190E042
S1132B4090937602809375028CE180937F0302E078
S1132B500093820310E11093810383E08093800348
S1132B60612F0E948B1D21E0F22EF09283030093CB
S1132B7086031093850396E0E92EE0928403612F87
S1132B808E2D0E948B1D89E08093870300938A0316
S1132B9010938903F0928803612F8F2D0E948B1D5F
S1132BA08BE180938B0300938E0310938D0385E058
S1132BB0F82EF0928C03612F8F2D0E948B1D8AE0DA
S1132BC080938F03009392031093910310929003C8
S1132BD0612F809190030E948B1D8FE1809393035A
S1132BE00093960310939503F0929403612F8F2D15
S1132BF00E948B1D8FE08093970300939A03109398
S1132C009903E0929803612F8E2D0E948B1D89E217
S1132C1080939B0300939E0310939D038CE0809309
S1132C209C03612F0E948B1D88E280939F03009375
S1132C30A2031093A1038BE08093A003612F0E9451
S1132C408B1D80E28093A3030093A6031093A50336
S1132C500093A403612F802F0E948B1D81E1809338
S1132C60A7030093AA031093A903B4E0FB2EF092E8
S1132C70A803612F8F2D0E948B1D8AE28093AB03E2
S1132C800093AE031093AD0387E08093AC03612FF0
S1132C900E948B1D0093AF030093B2031093B10302
S1132CA0F092B003612F8F2D25C68532910509F06E
S1132CB092C08AE090E09093290D8093280D80E1E2
S1132CC090E090937602809375028CE180937F0369
S1132CD0A2E0FA2EF092820310E11093810383E0C4
S1132CE080938003612F0E948B1D81E08093830376
S1132CF0F092860310938503F6E0EF2EE0928403AE
S1132D00612F8E2D0E948B1D8BE180938703F0929F
S1132D108A031093890305E000938803612F802FB1
S1132D200E948B1D8FE180938B03F0928E0310938E
S1132D308D0300938C03612F802F0E948B1D8FE0E5
S1132D4080938F03F092920310939103E092900387
S1132D50612F8E2D0E948B1D89E280939303F09244
S1132D609603109395038CE080939403612F0E9443
S1132D708B1D88E280939703F0929A031093990332
S1132D808BE080939803612F0E948B1D80E28093D7
S1132D909B03F0929E0310939D03F0929C03612F7A
S1132DA08F2D0E948B1D81E180939F03F092A203DB
S1132DB01093A10384E08093A003612F0E948B1DD4
S1132DC08AE28093A303F092A6031093A50387E0FD
S1132DD08093A4038EC58B31910509F0E4C085E08E
S1132DE090E09093290D8093280D80E190E09093DA
S1132DF076028093750285E180937F0302E000935D
S1132E00820310E1109381038DE080938003612F8E
S1132E100E948B1D85E280938303009386031093A5
S1132E208503EAE0FE2EF0928403612F8F2D0E9429
S1132E308B1D79E0D72ED092870300938A031093D9
S1132E40890361E0C62EC0928803612F8C2D0E94F5
S1132E508B1D00938B0300938E0310938D0354E01A
S1132E60E52EE0928C03612F8E2D0E948B1DF09233
S1132E708F03009392031093910310929003612F98
S1132E80809190030E948B1D86E2809393030093AC
S1132E9096031093950348E0F42EF0929403612F67
S1132EA08F2D0E948B1D1092970300939A03109309
S1132EB09903D0929803612F8D2D0E948B1D88E277
S1132EC080939B0300939E0310939D038BE0809358
S1132ED09C03612F0E948B1D81E180939F030093CB
S1132EE0A2031093A103E092A003612F8E2D0E94F0
S1132EF08B1D89E28093A3030093A6031093A5037B
S1132F008CE08093A403612F0E948B1D8BE280933D
S1132F10A7030093AA031093A9031092A803612F97
S1132F208091A8030E948B1D8FE08093AB030093D4
S1132F30AE031093AD0386E08093AC03612F0E942F
S1132F408B1D8AE28093AF030093B2031093B10305
S1132F5087E08093B003612F0E948B1D82E18093F0
S1132F60B3030093B6031093B503F092B403612F37
S1132F708F2D0E948B1D85E08093B7030093BA03C5
S1132F801093B903C092B803612F8C2D0E948B1D3E
S1132F9083E08093BB030093BE031093BD038EE0D4
S1132FA08093BC03A6C48632910509F083C088E0EF
S1132FB090E09093290D8093280D80E190E0909308
S1132FC07602809375028CE180937F0332E0F32EC6
S1132FD0F092820310E11093810383E080938003D5
S1132FE0612F0E948B1D8BE180938303F0928603F3
S1132FF01093850305E000938403612F802F0E94C2
S11330008B1D8FE180938703F0928A0310938903C9
S113301000938803612F802F0E948B1D8FE0809383
S11330208B03F0928E0310938D0386E080938C03C0
S1133030612F0E948B1D89E280938F03F09292038B
S1133040109391038CE080939003612F0E948B1D59
S113305088E280939303F0929603109395038BE098
S113306080939403612F0E948B1D80E280939703C9
S1133070F0929A0310939903F0929803612F8F2D85
S11330800E948B1D81E180939B03F0929E03109319
S11330909D0384E080939C03612F0E948B1D8AE230
S11330A080939F03F092A2031093A10387E080937F
S11330B0A0031FC4009709F0ADC089E090E090938D
S11330C0290D8093280D80E190E0909376028093FF
S11330D0750287E280937F0302E00093820310E18C
S11330E01093810300938003612F802F0E948B1D16
S11330F088E180938303009386031093850387E01C
S113310080938403612F0E948B1D89E08093870341
S113311000938A031093890321E0F22EF09288032E
S1133120612F8F2D0E948B1D9AE0E92EE0928B0374
S113313000938E0310938D0310928C03612F809162
S11331408C030E948B1D00938F03009392031093B2
S1133150910384E080939003612F0E948B1D8BE286
S11331608093930300939603109395031092940312
S1133170612F809194030E948B1D85E080939703B7
S113318000939A0310939903F0929803612F8F2D63
S11331900E948B1DF0929B0300939E0310939D034A
S11331A086E080939C03612F0E948B1D8CE18093A9
S11331B09F030093A2031093A10383E0F82EF092DF
S11331C0A003612F8F2D0E948B1D8EE08093A3039B
S11331D00093A6031093A503E092A403612F8E2D00
S11331E00E948B1D83E18093A7030093AA0310938D
S11331F0A903F092A803612F8F2D0E948B1D82E1F9
S11332008093AB030093AE031093AD0388E08093E7
S1133210AC036FC38F31910509F04CC085E090E099
S11332209093290D8093280D80E190E0909376028D
S11332308093750286E280937F03B2E0FB2EF092C6
S1133240820310E11093810388E080938003612F4F
S11332500E948B1D85E180938303F0928603109373
S113326085038DE080938403612F0E948B1D83E18D
S113327080938703F0928A031093890303E00093F9
S11332808803612F802F0E948B1D85E280938B031E
S1133290F0928E0310938D038AE080938C03612F48
S11332A00E948B1D00938F03F0929203109391035D
S11332B08EE0E9C28932910519F48CE090E026C2CF
S11332C08832910509F042C08BE090E09093290D7B
S11332D08093280D80E190E09093760280937502AC
S11332E082E180937F03A2E0FA2EF092820300E150
S11332F00093810318E010938003602F812F0E94B4
S11333008B1D86E280938303F092860300938503EA
S113331010938403602F812F0E948B1D85E180937D
S11333208703F0928A03009389038DE080938803D6
S1133330602F0E948B1D83E080938B03F0928E0399
S113334000938D038EE080938C03D3C28C3191055E
S113335009F069C083E090E09093290D8093280DD3
S113336080E190E0909376028093750285E18093EA
S11333707F0302E00093820310E1109381038DE048
S113338080938003612F0E948B1D85E280938303C9
S11333900093860310938503FAE0FF2EF0928403D2
S11333A0612F8F2D0E948B1DE9E0EE2EE0928703A2
S11333B000938A031093890381E080938803612F2B
S11333C00E948B1D00938B0300938E0310938D0337
S11333D084E080938C03612F0E948B1DF0928F03F5
S11333E0009392031093910310929003612F8091A4
S11333F090030E948B1D86E28093930300939603AF
S11334001093950388E080939403612F0E948B1D91
S11334101092970300939A0310939903E0929803F0
S1133420612F8E2D67C28F30910509F059C086E057
S113343090E09093290D8093280D80E190E0909383
S113344076028093750286E280937F0372E0E72E12
S1133450E092820310E11093810368E0D62ED092AB
S11334608003612F8D2D0E948B1D85E18093830342
S1133470E0928603109385038DE080938403612F8B
S11334800E948B1D83E180938703E0928A0310934B
S1133490890303E000938803612F802F0E948B1D12
S11334A05EE0F52EF0928B03E0928E0310938D0371
S11334B08AE080938C03612F0E948B1D82E18093AC
S11334C08F03E092920310939103D0929003612FA3
S11334D08D2D0E948B1D00939303E0929603BDC033
S11334E08131910509F05DC084E090E09093290D4D
S11334F08093280D80E190E090937602809375028A
S113350086E280937F0342E0F42EF092820310E17E
S11335101093810338E0E32EE0928003612F8E2D17
S11335200E948B1D85E180938303F09286031093A0
S113353085038DE080938403612F0E948B1D83E1BA
S113354080938703F0928A031093890303E0009326
S11335508803612F802F0E948B1D85E280938B034B
S1133560F0928E0310938D038AE080938C03612F75
S11335700E948B1D82E180938F03F092920310933B
S11335809103E0929003612F8E2D0E948B1D009376
S11335909303F0929603109395038EE08093940323
S11335A0A8C18032910509F05DC082E090E090935B
S11335B0290D8093280D80E190E09093760280930A
S11335C0750286E280937F0322E0D22ED09282039A
S11335D010E11093810388E080938003612F0E949F
S11335E08B1D85E180938303D0928603109385031A
S11335F08DE080938403612F0E948B1D85E280936C
S11336008703D0928A03109389039AE0E92EE0920B
S11336108803612F8E2D0E948B1D83E180938B0381
S1133620D0928E0310938D0303E000938C03612FDB
S1133630802F0E948B1D8EE0F82EF0928F03D09283
S1133640920310939103E0929003612F8E2D0E94B8
S11336508B1D00939303D092960310939503F092DD
S1133660940320CB8231910509F04BC088E090E0AF
S11336709093290D8093280D80E190E09093760239
S1133680809375028BE280937F0302E000938203B0
S113369010E11093810310928003612F80918003C5
S11336A00E948B1D81E18093830300938603109312
S11336B0850384E080938403612F0E948B1D8FE037
S11336C08093870300938A031093890386E0809391
S11336D08803612F0E948B1D10928B0300938E032D
S11336E010938D0389E080938C03612F0E948B1DBE
S11336F088E280938F0300939203109391038BE0ED
S1133700C2C08A32910589F587E090E09093290D33
S11337108093280D80E190E0909376028093750267
S113372086E280937F0302E00093820310E110930A
S1133730810388E080938003612F0E948B1D85E1C3
S11337408093830300938603109385038DE0809315
S11337508403612F0E948B1D83E080938703009371
S11337608A03109389038EE0C2C08B32910519F548
S11337701092290D1092280D80E190E0909376022A
S11337808093750282E180937F0302E000938203B9
S113379010E11093810388E080938003612F0E94DD
S11337A08B1D10928303009386031093850389E095
S11337B0809384039EC085309105C1F481E090E03C
S11337C09093290D8093280D80E190E090937602E8
S11337D08093750210927F0382E08093820390E1CC
S11337E09093810389E08093800383C083319105A2
S11337F009F04CC083E090E09093290D8093280D4C
S113380080E190E090937602809375028FE180933B
S11338107F0302E00093820310E11093810385E0AB
S113382080938003612F0E948B1D81E18093830329
S1133830009386031093850384E080938403612FAF
S11338400E948B1D8FE08093870300938A0310935B
S1133850890386E080938803612F0E948B1D80E298
S113386080938B0300938E0310938D0300938C033A
S1133870612F802F0E948B1D10928F03009392035F
S11338801093910389E08093900333C00E97A1F5C0
S11338908AE090E09093290D8093280D80E190E0D8
S11338A090937602809375028FE080937F0302E009
S11338B00093820310E11093810386E080938003D8
S11338C0612F0E948B1D80E2809383030093860303
S11338D01093850300938403612F802F0E948B1D16
S11338E01092870300938A031093890389E08093DD
S11338F0880360E10E948B1D80917502909176028D
S113390000912D0E10912E0E809F9001819F300DFD
S1133910909F300D11243093560B2093550B8091BA
S1133920DA039091DB03809F9001819F300D909F7B
S1133930300D112430932C0E20932B0EC801AA278E
S113394097FDA095BA2FBC01CD010E947B3017FFD3
S113395006C020E030E040E857E40E94CE2F2FE676
S113396032E143E85FE30E94EA30DC01CB01BC01B1
S1133970CD010E945E30DC01CB019093FB0A809361
S1133980FA0ACE0101960E94CC1D0B811C81C8014C
S1133990AA2797FDA095BA2FBC01CD010E947B30C8
S11339A017FF06C020E030E040E857E40E94CE2F25
S11339B025EE38E34EE054E40E94EA306B017C01CA
S11339C009811A81C801AA2797FDA095BA2FBC01C5
S11339D0CD010E947B3017FF06C020E030E040E8B4
S11339E057E40E94CE2F28EE38E34EE05CE30E94B9
S11339F0EA30DC01CB019C01AD01C701B6010E9494
S1133A00CE2FDC01CB01BC01CD010E945E305B01F5
S1133A106C0180902D0E90902E0E740100271127BA
S1133A20A80197010E947731DC01CB01A80197011D
S1133A30281B390B4A0B5B0B57FD05C0CA01B901A2
S1133A400E947B3016C0DA01C90181709070A070A9
S1133A50B0705695479537952795822B932BA42BB9
S1133A60B52BBC01CD010E947B309B01AC010E94AF
S1133A70CE2F2FE632E143E85FE30E94EA30DC0117
S1133A80CB01BC01CD010E945E307B018C0194010D
S1133A9044275527C601B5010E9477312093410D73
S1133AA03093420D4093430D5093440D8091750221
S1133AB09091760201972091410D3091420D82231D
S1133AC0932390932E0D80932D0D8091DA03909182
S1133AD0DB030197282339233093D8032093D7039A
S1133AE0A801970161E086E00E94670881E090E008
S1133AF024960FB6F894DEBF0FBECDBFDF91CF91F1
S1133B001F910F91FF90EF90DF90CF90BF90AF90F7
S1133B109F908F9008950F931F93CF93282F162F64
S1133B208FB7F894082F862F99276091DA03709144
S1133B30DB036817790758F1C22FE22FFF27E61736
S1133B40F70728F52091570B3091580B4091590BEA
S1133B5050915A0B81E090E0A0E0B0E004C0880FDF
S1133B60991FAA1FBB1FEA95D2F7282B392B4A2B82
S1133B705B2BC10FEC2FFF27E617F70758F32093B1
S1133B80570B3093580B4093590B50935A0B0FBF5C
S1133B90CF911F910F910895FC018FB7F894282FAE
S1133BA0332780918800909189008083918380914C
S1133BB07C0084FF0EC08091180290911902019636
S1133BC0909319028093180280917C008061809305
S1133BD07C008091180290911902828393832FBFF5
S1133BE008958F929F92AF92BF92CF92DF92EF92FD
S1133BF0FF920F931F93CF93DF93CDB7DEB7C054DB
S1133C00D0400FB6F894DEBF0FBECDBF6196EEACC8
S1133C10FFAC61976396CEACDFAC639773E5A72ED8
S1133C20B12CAC0EBD1ED601ED916D01E53261F0F3
S1133C30EE2309F494C0D701ED937D011C92D601C3
S1133C40ED916D01E532A1F720E0D601ED916D0112
S1133C508E2F99278F369105B1F18037910574F431
S1133C6083369105C9F08436910524F48335910592
S1133C70F1F018C08936910579F114C085379105A2
S1133C8061F18637910524F48337910581F00AC0E8
S1133C908837910531F106C0F50182E090E0A80E65
S1133CA0B91EE081D701ED937D011C92BCCFF501D3
S1133CB082E090E0A80EB91E00811181B801C7010D
S1133CC00E94C22FB0CF68E0862E912C80E3D701EA
S1133CD08D937D012C9308C021E05AE0852E912C10
S1133CE003C040E1842E912CF50182E090E0A80EFF
S1133CF0B91E0190F081E02D222351F0F7FF08C096
S1133D00F095E195FF4F8DE2D7018D937D011C92D3
S1133D108E010F5B1F4FD8011E928D01CF01B4019C
S1133D200E946331282F205D2A330CF0295DD801CD
S1133D302E938D01CF01B4010E946331FB01672BE7
S1133D4069F7B801C7010E94C22FF8010190002051
S1133D50E9F73197E01BF10BEE0EFF1E64CF80E014
S1133D6090E0C05CDF4F0FB6F894DEBF0FBECDBF4E
S1133D70DF91CF911F910F91FF90EF90DF90CF9043
S1133D80BF90AF909F908F900895CF93DF938AE078
S1133D900E94DA1E809177028A3049F0C6E7D2E0A9
S1133DA0219688810E94DA1E89818A30C9F7DF91C1
S1133DB0CF910895CF93C82F8A3019F48DE00E94D3
S1133DC0DA1E5D9BFECFCCB9CF9108958F929F925E
S1133DD0AF92BF92CF92DF92EF92FF920F931F9315
S1133DE0CF93DF93CDB7DEB72C970FB6F894DEBF31
S1133DF00FBECDBF682F8091260E811160958091F2
S1133E00680299278430910509F46FC285309105C1
S1133E105CF48230910509F4EAC4833091050CF016
S1133E20E4C1019769F0E3C48630910509F4D9C26D
S1133E30863091050CF47DC2079709F483C4D7C476
S1133E402091660D8FB7F89499272093BC0A8FBFF1
S1133E504091280E5091290E4F5F5F4F5093290EC9
S1133E604093280E8091540199278530910509F4D7
S1133E70F7C08630910554F483309105C1F1843044
S1133E8091050CF06CC0029769F08BC187309105E5
S1133E9009F424C1873091050CF4FBC0089709F498
S1133EA047C17FC18091CF039091D0030196909335
S1133EB0D0038093CF038091D1039091D20348170C
S1133EC0590780F4E091BF0DF091C00DE35BFF4F03
S1133ED0808191818F5F9F4F09F089C448305105DB
S1133EE008F485C483E38093660D83E057C1809111
S1133EF0CF039091D00301969093D0038093CF0386
S1133F008CEC8093660D84E0809354018FEF9FEFD7
S1133F109093290E8093280EE090BF0DF090C00D71
S1133F20F70182818F3D09F062C487010B5F1F4F47
S1133F30CE0101960E94CC1D8B819C81F701858363
S1133F40968389819A81F8018283938381E08483B3
S1133F5080910001909101018583968348C48091EA
S1133F60CF039091D00301969093D0038093CF0315
S1133F708091280E282F33278091DE039091DF0350
S1133F802817390708F066C0E091BF0DF091C00D05
S1133F9082818F3DE1F545305105C9F5A5E0EA2E52
S1133FA0F12CEE0EFF1E6E010894C11CD11CC6013B
S1133FB00E94CC1D8091D3039091D40329813A812E
S1133FC0B901680F791F4B815C81E091D503F091B1
S1133FD0D603809590958217930748F46F5F7F4FBF
S1133FE069837A834E0F5F1F4F5F5F4F04C06983FD
S1133FF07A834E0F5F1F4B835C83F601828193812A
S1134000F7018083918389819A8182839383E091EC
S1134010BF0DF091C00D8091280E9091290EE80FEC
S1134020F91F20812093660D8091630A9091640AA0
S1134030EAE6F1E02927220FF11DE20FF11DC895F0
S1134040982F802D3196C89590259093640A80937B
S1134050630ACDC38091630A8093660D85E09EC098
S11340608091CF039091D00301969093D0038093D5
S1134070CF038091630A9091640A892F99278093D2
S1134080660D86E0809354011092290E1092280E3A
S1134090AEC38091CF039091D00301969093D00347
S11340A08093CF034430510508F4A1C31092290E24
S11340B01092280E80910D0D882311F087E06EC0B8
S11340C08091F30A9091F40A01969093F40A8093F4
S11340D0F30ABB98BA980E9448085FC04130510562
S11340E071F48091CF039091D00301969093D00303
S11340F08093CF03BB98BA980E94480878C38091F4
S1134100330E9091340E01969093340E8093330EB7
S11341104430510508F46BC388E080935401109235
S1134120290E1092280E1092A10E1092A00E5FC3B9
S11341308091330E9091340E01969093340E8093B7
S1134140330E20E08091A00E9091A10E880F991F4C
S11341509093A10E8093A00E67FF05C08160909399
S1134160A10E8093A00E660F8091A00E9091A10ED7
S113417083589A4B09F423C32F5F283018F3809196
S1134180280E9091290E429708F431C3E091BF0D97
S1134190F091C00DE15BFF4F108289E080935401E0
S11341A026C310921A02E091BF0DF091C00D8281D6
S11341B08E5D823020F48091C10D80930D0D88E7CF
S11341C099E20E940303882309F411C323E0209396
S11341D068028091150D9091160D01969093160D1D
S11341E08093150D20936D02A4C28091330E90919B
S11341F0340E01969093340E8093330E6A3A11F084
S1134200653521F58091950E9091960E01969093C7
S1134210960E8093950E039708F4E9C210928C0EC3
S11342201092960E1092950E1092F20A1092F10AC4
S11342301092E0031092640A1092630A8BE490E0F7
S11342409093100D80930F0D85E070C080910C0247
S1134250882359F180911E0D882339F181E090E083
S1134260A0E0B0E000902D0D04C0880F991FAA1F94
S1134270BB1F0A94D2F72FB7F894622F2091570BE3
S11342803091580B4091590B50915A0B8223932330
S1134290A423B5230097A105B10511F081E001C065
S11342A080E06FBF882309F0A2C280911A0288239C
S11342B009F49DC28091340D9091350D019790932E
S11342C0350D8093340D181619060CF490C284E051
S11342D08093680280936D0210925E0D10929A0E84
S11342E01092960E1092950E24C28091330E9091E6
S11342F0340E01969093340E8093330E6A3A19F07B
S1134300653509F074C280915C0D90915D0D019644
S113431090935D0D80935C0D0E94800A8F70907065
S113432001969093350D8093340D83E08093680259
S11343305EC28091330E9091340E01969093340EA8
S11343408093330E6A3A11F0653519F460935B0A71
S11343504EC280918C0E9927009719F00697C4F5E8
S113436003C060935A0A37C020915A0A30915B0AFD
S1134370922F882790935B0A80935A0A60935A0A73
S1134380FF24220F331F67FD2160660F83E32C3C5B
S11343903807C9F4E091240DF091250D94819923F7
S11343A0B9F486E08093680280936D028FB7F89425
S11343B0082F1127892F0E944C130FBF87E08F19F4
S11343C08093E00308C0F394E7E0EF15D0F603C050
S11343D083E08093680280918C0E8F5F80938C0EB3
S11343E006C28091330E9091340E01969093340E50
S11343F08093330E80915A0A90915B0A982F8827F4
S113440090935B0A80935A0A60935A0A20915A0A3D
S113441030915B0A0090E00302C0369527950A9418
S1134420E2F7F22EE091240DF091250D8091F10A2E
S11344309091F20AE80FF91F20834091F10A5091FC
S1134440F20A4F5F5F4F5093F20A4093F10A809152
S11344500F0D9091100D4817590788F58091630A44
S11344609091640AEAE6F1E0F926FF0CF11DEF0DE4
S1134470F11DC895982F802D3196C895902590935D
S1134480640A8093630A4530510509F0B0C1E09194
S1134490240DF091250D848199279093100D80931C
S11344A00F0D8734910528F0148283E0809368020D
S11344B0FBC105969093100D80930F0D98C148177A
S11344C0590709F0B1C0A091240DB091250D1296A1
S11344D08C9112978F3D09F08BC08FB7F894E82E1A
S11344E09D012B5F3F4F05E0802E912C8C0E9D1E6D
S11344F015968D919C9116978F839887F9018281E7
S113450093818D839E838481C82EDD248581968149
S1134510909307028093060219E0A12EB12CAC0EF1
S1134520BD1EC5010E94CC1D2F8138858B859C85BD
S11345308217930750F02817390760F02D813E81C8
S113454089859A858217930710F401E006C028171D
S1134550390710F402E001C003E0013019F4A501A9
S1134560B40104C0023039F4A401B5018FE59DE023
S11345700E94692408C01092600D10925F0DEFE54F
S1134580FDE0128213820093470DC114D10419F483
S1134590B1E0CB2ED12CF8E0CF16D10440F560E089
S11345A070E06C157D0518F52091610D3091620D58
S11345B080915F0D9091600DA901569547956F5FAD
S11345C07F4F20FF06C09A019695879581509048A9
S11345D003C09A01969587956C157D0568F39093B1
S11345E0600D80935F0D3093620D2093610DEFBEDB
S11345F08091630A9091640AEAE6F1E0F926FF0CDF
S1134600F11DEF0DF11DC895982F802D3196C89599
S113461090259093640A8093630A8BE490E09093CE
S1134620F20A8093F10AE3C04D34510508F4DFC067
S1134630A091240DB091250DFD01E55BFF4F208174
S113464031818091630A9091640A28173907A9F58A
S113465012968C918F3D21F48EE599E20E9403031A
S1134660E091240DF091250DE55BFF4F81E090E092
S113467080839183EB54F04080910D0D8823F9F0F1
S1134680208131818091000190910101281739071F
S1134690B1F487E0809368020E941D13BB9ABA9A12
S11346A08FB7F894282F33278AEA8093BC0A2FBF48
S11346B01092F20A1092F10AF7C0108211820E943D
S11346C0981383E08093680280910C02813071F426
S11346D080911A02882351F08091340D9091350D08
S11346E00E94F00F9093350D8093340DE091240DCA
S11346F0F091250DE35BFF4F8091360D9091370DBE
S11347008083918382E994E20E940303882369F4FD
S1134710E091240DF091250D848383E08093680259
S113472080EC8DB9B8980E94D70880916802809374
S11347306D028FB7F894082F112780E00E944C1364
S11347400FBF55C08091CF039091D00301969093F1
S1134750D0038093CF03E091F10AF091F20A3196ED
S1134760F093F20AE093F10AE031F105A0F10E941E
S11347704808BB98BA980E94981303E00093680213
S1134780E091240DF091250DE35BFF4F8091360DF0
S11347909091370D8083918382E994E20E94030310
S11347A0882329F5E091240DF091250D848300934D
S11347B0680280EC8DB9B8980E94D70818C0E091BF
S11347C0BF0DF091C00DE15BFF4F81E0808389E074
S11347D08093540169C0EB30F10548F0E850FF4F75
S11347E020818FB7F89499272093BC0A8FBF20911A
S11347F01C0D30911D0D25363105C0F08091570DEB
S11348009091580D01969093580D8093570D809177
S1134810040290910502019690930502809304028C
S11348202456304030931D0D20931C0D2091CF034E
S11348303091D00325363105C0F08091570D909109
S1134840580D01969093580D8093570D80912B0D20
S113485090912C0D019690932C0D80932B0D245642
S113486030403093D0032093CF032091330E309106
S1134870340E25363105C0F08091570D9091580DB6
S113488001969093580D8093570D8091F60A90915C
S1134890F70A01969093F70A8093F60A245630405B
S11348A03093340E2093330E81E090E02C960FB6B3
S11348B0F894DEBF0FBECDBFDF91CF911F910F9152
S11348C0FF90EF90DF90CF90BF90AF909F908F902C
S11348D00895CF93DF93EC01FB01DA018D919C9154
S11348E01197208131814281538112966D917C917F
S11348F013972817390758F4821B930B80959095CA
S113490088839983461B570B4150504006C0281B8F
S1134910390B28833983461B570B4A835B83DF910A
S1134920CF9108951F93CF93DF938FB7F894182FE7
S11349308091150D9091160D8536910570F080913A
S11349400D0D8093C10D10920D0D85E69AE00E9425
S1134950660F1092160D1092150D8091150D909101
S1134960160D01969093160D8093150D2091240D2C
S11349703091250D205B3F4FF901108211822055A3
S11349803040E901D901159660910C02613009F0BB
S113499063C080917803882309F45EC08A818E3DC8
S11349A009F05AC0C55BDF4F88819981CB54D04050
S11349B0892B09F451C013968D919C9114974091C1
S11349C00001509101018417950709F445C08D81B8
S11349D0882339F511962D913C91129724173507A8
S11349E001F56093700D80912F0D9091300D90938F
S11349F0720D8093710D3093740D2093730D90910B
S1134A000B02992359F480910D0D8093C10D90935D
S1134A100D0D8BE69DE00E94660F27C06093520B3C
S1134A2024C08C91813009F580931E0D13962D912D
S1134A303C91149780912F0D9091300D28173907D0
S1134A40A1F41092310E1092240E1092230E1092A3
S1134A5056011092550109C0F90182818E5D8230A0
S1134A6020F0C9010E94A30AEC01209721F0D09301
S1134A70250DC093240DE091240DF091250D148291
S1134A801FBF80EC8DB9B8980E94D708DF91CF91F1
S1134A901F91089578941F920F920FB60F921124CC
S1134AA06F927F928F929F92AF92BF92CF92DF923A
S1134AB0EF92FF920F931F932F933F934F935F9324
S1134AC06F937F938F939F93AF93BF93EF93FF93D2
S1134AD0CF93DF93CDB7DEB72497F894DEBF7894F5
S1134AE0CDBF80917A03882309F4F4C08091450DE9
S1134AF08230A9F48091670D9091680D809590950E
S1134B0090938900809388008091180290911902F3
S1134B102091690D30916A0D821B930B15C0813071
S1134B20B9F48091670D9091680D909389008093FA
S1134B30880080911802909119022091690D30919A
S1134B406A0D820F931F01969093190280931802A5
S1134B5010927A0380917703882309F4C4C0CE01AC
S1134B6001960E94CC1D0B811C81C801AA2797FDC8
S1134B70A095BA2FBC01CD010E947B3017FF06C05F
S1134B8020E030E040E857E40E94CE2F25EE38E3E1
S1134B904EE054E40E94EA306B017C0109811A81E1
S1134BA0C801AA2797FDA095BA2FBC01CD010E9488
S1134BB07B3017FF06C020E030E040E857E40E9455
S1134BC0CE2F28EE38E34EE05CE30E94EA30DC01AD
S1134BD0CB019C01AD01C701B6010E94CE2FDC01BF
S1134BE0CB01BC01CD010E945E304B015C016090A1
S1134BF02D0E70902E0E730100271127A801970126
S1134C000E947731DC01CB01A8019701281B390BE5
S1134C104A0B5B0B57FD05C0CA01B9010E947B30EA
S1134C2016C0DA01C90181709070A070B0705695F9
S1134C30479537952795822B932BA42BB52BBC0135
S1134C40CD010E947B309B01AC010E94CE2F2FE648
S1134C5032E143E85FE30E94EA30DC01CB01BC01AE
S1134C60CD010E945E306B017C01930144275527DE
S1134C70C501B4010E9477312093410D3093420D58
S1134C804093430D5093440D8091750290917602A8
S1134C9001972091410D3091420D822393239093EB
S1134CA02E0D80932D0D8091DA039091DB030197F3
S1134CB0282339233093D8032093D70360910C021F
S1134CC0613029F4A701960186E00E9467081092DA
S1134CD0770309C08091180290911902019690936C
S1134CE01902809318022496F894DEBFCDBFDF9199
S1134CF0CF91FF91EF91BF91AF919F918F917F9150
S1134D006F915F914F913F912F911F910F91FF9060
S1134D10EF90DF90CF90BF90AF909F908F907F9057
S1134D206F900F900FBE0F901F901895382F8091A1
S1134D30CE0D99278230910509F46BC0833091051B
S1134D402CF4009759F0019781F1B7C18330910594
S1134D5009F49CC0049709F459C1AFC13E3709F066
S1134D60AEC180913D0D9927FC01EE0FFF1FEE0FA0
S1134D70FF1FE80FF91FE80FF91FE55BF24F82816F
S1134D809381009709F09BC111829093610A8093EB
S1134D90600A90937E0380937D0384819581909330
S1134DA0650D8093640D81E085C13E3709F487C1A8
S1134DB080913D0D9927FC01EE0FFF1FEE0FFF1FA1
S1134DC0E80FF91FE80FF91FE55BF24F308380917C
S1134DD0600A9091610AEAE6F1E0232F2927220F65
S1134DE0F11DE20FF11DC895982F802D3196C895BD
S1134DF090259093610A8093600A832F99278134C8
S1134E00910529F08234910509F453C156C182E019
S1134E1051C13E3709F451C160913D0D3D3781F4D4
S1134E20862F9927FC01EE0FFF1FEE0FFF1FE80FDF
S1134E30F91FE80FF91FE55BF24F80E281833FC160
S1134E40862F9927FC01EE0FFF1FEE0FFF1FE80FBF
S1134E50F91FE80FF91FE55BF24F21812327218316
S1134E608091600A9091610AEAE6F1E02927220F15
S1134E70F11DE20FF11DC895982F802D3196C8952C
S1134E8090259093610A8093600A13C140917D0339
S1134E9050917E034535510508F0BAC03D3711F4F1
S1134EA084E008C13E3709F07FC04230510508F460
S1134EB05FC0E091640DF091650DE40FF51F8291E0
S1134EC09927382F222782919927282B392B8091D3
S1134ED0600A9091610A60913D0D28173907E1F449
S1134EE0862F9927FC01EE0FFF1FEE0FFF1FE80F1F
S1134EF0F91FE80FF91FE55BF24F4250504042831F
S1134F0053838CE09BE20E94030380913D0D8F5FED
S1134F10817080933D0D10C0862F9927FC01EE0F00
S1134F20FF1FEE0FFF1FE80FF91FE80FF91FE55BE6
S1134F30F24F12821382118280913D0D9927FC0158
S1134F40EE0FFF1FEE0FFF1FE80FF91FE80FF91F09
S1134F50E55BF24F82819381892BD9F48481958119
S1134F609093650D8093640D81E08093CE0D13C002
S1134F7080913D0D9927FC01EE0FFF1FEE0FFF1FDF
S1134F80E80FF91FE80FF91FE55BF24F1282138255
S1134F9011821092CE0D1092610A1092600A109242
S1134FA07E0310927D038BC0E091640DF091650D3A
S1134FB0E40FF51F308340917D0350917E0342300E
S1134FC05105E8F02091600A3091610AE091640D86
S1134FD0F091650DE40FF51F32978081EAE6F1E068
S1134FE08327880FF11DE80FF11DC895322F202D5E
S1134FF03196C89530253093610A2093600A4F5F3B
S11350005F4F50937E0340937D0359C03E37D1F4E4
S11350101092610A1092600A10927E0310927D032E
S113502080913D0D9927FC01EE0FFF1FEE0FFF1F2E
S1135030E80FF91FE80FF91FE55BF24F12821382A4
S113504011823BC080E28327E091640DF091650DED
S113505020917D0330917E03E20FF31F8083409102
S11350607D0350917E0342305105E8F02091600A9F
S11350703091610AE091640DF091650DE40FF51F24
S113508032978081EAE6F1E08327880FF11DE80F6B
S1135090F11DC895322F202D3196C89530253093B7
S11350A0610A2093600A4F5F5F4F50937E034093E1
S11350B07D0383E08093CE0D02C01092CE0D81E07B
S11350C090E008958FB7F89499272091330D1092AA
S11350D0330D8FBF222309F4A4C08091250E87309D
S11350E031F41092250E8DE99EE00E94030321E025
S11350F08091250E99278430910509F46EC085307E
S1135100910554F48230910561F1833091050CF0DE
S113511058C0019749F07CC08630910509F471C0EC
S113512006970CF463C074C082E08093250E20912E
S113513057013091580180910902EAE6F1E0832792
S1135140880FF11DE80FF11DC895322F202D3196DF
S1135150C895302530935801209357018091090256
S113516054C0E091EE0AF091EF0A2091130D3091B2
S1135170140DE20FF31F5081809157019091580153
S1135180EAE6F1E0452F4927440FF11DE40FF11D34
S1135190C895982F802D3196C895902590935801E5
S11351A0809357012F5F3F4F3093140D2093130DBD
S11351B080916B0290916C022817390798F084E073
S11351C00FC08091320E90E289270E94840E282F0E
S11351D080915B0D8093250E1BC05091570185E093
S11351E08093250E852F0E94142911C080915701A8
S11351F090915801292F332786E08093250E822F22
S1135200F2CF87E08093250E8EE70E94840E282F2C
S1135210213039F088E08093250E8DE99EE00E94CC
S1135220030381E090E00895982F8D57823078F43D
S11352308FB7F894282F33278091250E80935B0D28
S113524083E08093250E9093320E2FBF9DE7892F24
S11352500E94840E992708958FBF08958FB7F894FC
S113526099270895E0913E0DF0913F0D8081918141
S11352708E379105B1F461E08FB7F89490919D0E4B
S113528092FD08C0946090939D0EF0930202E09307
S1135290010201C060E08FBF613039F40E941C0E2E
S11352A003C0CF010E94660F682F662331F48091FA
S11352B03E0D90913F0D0E94D70E089521E020935A
S11352C077038091470D8093450D8091610D9091F6
S11352D0620D90936A0D8093690D80915F0D90919A
S11352E0600D9093680D8093670D20937A03089561
S11352F08FB7F8949927E091BF0DF091C00DE05B52
S1135300FF4F10821182E055F0408FBF82818E5D85
S1135310823020F061E0CF010E94D70E8FB7F8945D
S1135320992710920B028FBF8091150D9091160D45
S113533085369105A0F08FB7F894282F33278091F4
S11353400D0D8093C10D10920D0D2FBF85E69AE0CF
S11353500E94660F1092160D1092150D08959091EB
S11353600C029130D1F48091520B8130B1F48FB79B
S1135370F894282F332780910D0D8093C10D10923E
S11353800D0D2FBF8BE69DE00E94660F8FB7F8943A
S113539099271092520B8FBF0895913009F580918F
S11353A0310E8130E9F48FB7F894282F3327809198
S11353B00D0D8093C10D10920D0D2FBF88EB9CE055
S11353C00E94660F8FB7F89499271092310E8FBF01
S11353D08FB7F89499271092240E1092230E8FBF42
S11353E008958091310D9091320DAA27BB279C011D
S11353F0AD0161E085E00E94670808959F92AF9235
S1135400BF92CF92DF92EF92FF920F931F93CF93AD
S1135410DF9381E08093270D8FB7F8949927C0908C
S11354201A0DD0901B0D10921B0D10921A0D8FBFE8
S113543080918D0E90918E0EA0918F0EB091900E52
S11354400097A105B10509F495C09924CDE7DBE0E7
S1135450AA24BB2451E0E52EF12C012D112D0A2C98
S113546004C0EE0CFF1C001F111F0A94D2F7809198
S11354708D0E90918E0EA0918F0EB091900E8E2174
S11354809F21A023B1230097A105B10509F469C0A8
S11354909601442755278D819E81AF81B885821B53
S11354A0930BA40BB50B8D839E83AF83B8870397AF
S11354B0A105B1050CF055C086E89BE20E940303E8
S11354C0882309F445C08881882389F48D819E81CD
S11354D0AF81B88529813A814B815C81820F931F0A
S11354E0A41FB51F8D839E83AF83B8871AC0A801FC
S11354F09701209530954095509580918D0E90910F
S11355008E0EA0918F0EB091900E82239323A4232C
S1135510B52380938D0E90938E0EA0938F0EB0932F
S1135520900E8091990E893019F48FEF8093990E23
S11355309091990E9F5F9093990E8091470A8F5F87
S11355408093470AE92FFF27E25FFD4F908209C04D
S11355508091490D9927AA27BB278D839E83AF830A
S1135560B88793940894A11CB11C299689E08915E5
S113557008F070CF8FB7F8949927C0901A0DD09087
S11355801B0D8FBFCD2811F40E942402DF91CF910F
S11355901F910F91FF90EF90DF90CF90BF90AF904D
S11355A09F90089587B799278C7F009719F080E022
S11355B090E01AC06F9918C0379B03C088E090E050
S11355C013C087B7992783709070892B59F081B7DE
S11355D092B7891B803118F48CE190E005C088E112
S11355E090E002C080E190E0382F8093080225B754
S11355F0237E8C3121F0883111F008C0000080B77F
S1135600992787709070892BC9F7237E232B25BF98
S113561085B7806285BF08950F931F93CF93DF935F
S11356209091270E86E0989F80011124055B124F0C
S1135630F801C481D581828193810597C0F12081CD
S1135640822F99278134910559F08234910524F4ED
S11356508034910561F125C08234910591F021C017
S1135660C55BDF4F81E090E088839983CB54D040C1
S1135670F80181818093480D80E79BE20E94030337
S113568008C0C55BDF4F81E090E088839983CB54E9
S1135690D040809102018B83CE010E94A30AEC01C9
S11356A006C0209361028DE09FE20E9403038FB73E
S11356B0F894282F3327209719F0F801C483D58351
S11356C0F8011282138211828091270E8F5F8170FC
S11356D08093270E2FBFDF91CF911F910F910895D3
S11356E02091480D31E08FB7F89490919D0E91FD73
S11356F006C0926090939D0E2093400D01C030E04F
S11357008FBF313011F40E941C0E08958F929F9226
S1135710AF92BF92CF92DF92EF92FF920F931F93BB
S1135720CF93DF939091470A992319F48AE090E08C
S113573015C080910302893019F48FEF809303021E
S1135740809103028F5F8093030291509093470AE4
S1135750E82FFF27E25FFD4F808199278A3008F008
S11357604FC399278430910509F455C185309105BB
S113577094F48130910509F453C0823091051CF4EE
S1135780892B01F13DC38230910509F4FEC00397D2
S113579009F434C135C38730910509F427C388302F
S11357A0910544F48530910509F44DC1069709F437
S11357B0FFC126C38830910509F41BC3099709F476
S11357C01BC31EC31092D903809100019091010163
S11357D0009729F422E330E0AC0160E018C028EE21
S11357E033E040E050E060E082E00E946708E0912E
S11357F06902F0916A02309719F06081718102C0E8
S11358006FEF7FEF22E330E040E050E0CA010E94F6
S1135810F81320E038E240E050E060E081E0C5C1E8
S1135820E091D903EE2309F08FC080917B03882394
S113583009F48AC080915D0A90915E0A0196909362
S11358405E0A80935D0ACE2F7EE2C72E72E0D72EC9
S1135850EE24FF24F60181916F018823F9F01FB72C
S11358601078F89499279F938F93FF92EF9289E091
S113587091E09F938F9387E792E09F938F930E9489
S1135880F11D8DB79EB708960FB6F8949EBF0FBE54
S11358908DBF0E94C51E112309F07894CF5F089430
S11358A0E11CF11CC233B0F21FB71078F894809158
S11358B00402909105022091F60A3091F70A409172
S11358C02B0D50912C0D60912F0E7091300E9F93E3
S11358D08F933F932F935F934F937F936F93809115
S11358E0200D9091210D9F938F9388E191E09F93D8
S11358F08F9387E792E09F938F930E94F11DEDB7FA
S1135900FEB73E960FB6F894FEBF0FBEEDBF0E94E1
S1135910C51E112309F078941092210D1092200DC8
S11359201092390D1092380D0E9429081092300EF1
S113593010922F0EC0E0EC2FFF27E25DFD4F108286
S1135940CF5FC233C0F35CC2EE2309F459C2809125
S11359507B03882309F454C28091000190910101D2
S1135960892B41F028EE33E040E050E060E082E033
S11359700E94670820E038E240E050E060E081E007
S11359800E9467081092D9033BC28091350E882388
S113599009F036C280917B03882309F431C28091D7
S11359A00001909101019093D70D8093D60D9093AF
S11359B0D50D8093D40D8FEF8093DA0D6DE48FECC9
S11359C09DE00E94B70C813069F48091CF0D9091D5
S11359D0D00D2FEC3DE04CE1BC018DE40E94780D2C
S11359E0813019F080E090E002C081E090E09927D6
S11359F0813009F005C28093350E02C28091450AB8
S1135A009091460A90936702809366021092460A28
S1135A101092450AF5C18FB7F8949927209168022E
S1135A208FBF233009F0ECC18FB7F89499272093E6
S1135A306D028FBF8FB7F894082F112780E00E9462
S1135A404C130FBFDDC18091460D882309F4D8C1E2
S1135A508FB7F8949927209168028FBF3327283095
S1135A603105D9F12930310524F42330310531F0E1
S1135A7096C02930310509F455C091C0C0911A026D
S1135A80CC2311F58FB7F894082F112788E0809361
S1135A9068020E9498130FBF8091310D9091320DCE
S1135AA0AA27BB279C01AD0161E085E00E9467083D
S1135AB084E00E942C106FE38C2F0E9487076C2FC8
S1135AC08BE00E9487079CC18091310D9091320D2B
S1135AD0AA27BB279C01AD0166C08FB7F894282F75
S1135AE0332789E0809368022FBF10920D026BE385
S1135AF080E00E94870769E380E00E94870788ECC2
S1135B0090E0000000000000000000000000000021
S1135B100000019718161906A4F321E030E040E0D4
S1135B2050E041C00E9448088FB7F894082F11270D
S1135B3080E00E944C130FBF882389F422E330E0F5
S1135B4040E050E061E085E00E9467088FB7F89478
S1135B50282F332788E0809368022FBF0EC080E58A
S1135B6090E00000000000000000000000000000C1
S1135B700000019718161906A4F36FE380E00E9451
S1135B80870760E08BE00E94870780911C0D90914D
S1135B901D0D019690931D0D80931C0D31C125E0C0
S1135BA030E040E050E061E085E00E94670828C1F1
S1135BB061E0962E8091FA0A9091FB0AAA27BB27EE
S1135BC09C01AD01692D86E00E9467088091410D1A
S1135BD09091420DA091430DB091440D0196A11DE9
S1135BE0B11D8093410D9093420DA093430DB0934A
S1135BF0440D8FB7F894992790920C028FBF8FB7FA
S1135C00F894882E809175029091760201972091E4
S1135C10410D3091420D8223932390932E0D809356
S1135C202D0D8091DA039091DB030197282339230A
S1135C303093D8032093D70380917803882309F401
S1135C40C5C0A090230EB090240E0894A11CB11CD2
S1135C50B092240EA092230E80915501909156018A
S1135C60019690935601809355018091110D909166
S1135C70120D01969093120D8093110DC091F30AA9
S1135C80D091F40ACB30D10508F48FC0409708F4C2
S1135C908CC000915C0D10915D0DC801AA2797FD81
S1135CA0A095BA2FBC01CD010E947B306B017C0111
S1135CB017FF08C020E030E040E857E40E94CE2FF0
S1135CC06B017C01CE01AA2797FDA095BA2FBC01D8
S1135CD0CD010E947B30D7FF06C020E030E040E8D1
S1135CE057E40E94CE2F9B01AC01C701B6010E946C
S1135CF01830DC01CB0120E030E040E85EE3BC0179
S1135D00CD010E94EA307B018C0180916202909166
S1135D106302A0916402B091650220E030E040E4A7
S1135D205FE3BC01CD010E94EA30DC01CB019C01A0
S1135D30AD01C801B7010E94CE2FDC01CB018093D5
S1135D40620290936302A0936402B093650210927E
S1135D50120D1092110D10925D0D10925C0D1092A7
S1135D60F40A1092F30A20E030E040E450E4BC016D
S1135D70CD010E9488301816C4F4F0E6AF16B104C1
S1135D80A0F090921E0D1092560110925501809130
S1135D902F0D9091300D9093BF0C8093BE0C809189
S1135DA0620A882311F49092310E80911E0D88238B
S1135DB069F08091550190915601803C910530F035
S1135DC08091620A882311F480931E0D80911A0237
S1135DD0882351F08091340D9091350D0E94F00F7D
S1135DE09093350D8093340D8FBE0AC085EB9FE2EE
S1135DF005C089EE98E002C08AE19FE20E94030395
S1135E00DF91CF911F910F91FF90EF90DF90CF9092
S1135E10BF90AF909F908F9008958FB7F894282FDC
S1135E20332780919D0E886080939D0E2FBF0E9422
S1135E301C0E0895EF92FF920F931F93CF93DF935D
S1135E40CDE3DEE067E0E62EF12CEC0EFD1E1CE057
S1135E5000E080913C0D882309F080C07AE3872F0D
S1135E6063E00E945731782FE0916902F0916A0251
S1135E70309719F08081918102C08FEF90E0909368
S1135E80450E8093440E8091170D9091180DF701E3
S1135E908283938330E0632F3717B8F54091B90AB2
S1135EA0862F840F282F2F5F203108F02051822F56
S1135EB09927DC0154E0AA0FBB1F5A95E1F7A80FFC
S1135EC0B91FA80FB91FAF5DB64F1D968C911D97D2
S1135ED080FF16C050965C915097553688F0832FFA
S1135EE09927FC01EE0FFF1FE80FF91FEC5BF14F40
S1135EF08D919C918583968357833F5F1D5F022F0D
S1135F006F5F603110F4371758F20093B90AF70144
S1135F10348380910001909101018A839B83909343
S1135F203E0E80933D0E8091260D8E838091410A12
S1135F309091420A8C839D8301969093420A8093A8
S1135F40410A28E33EE0412F6FEF7FEF8AEF0E9482
S1135F50780D9927813011F480933C0DDF91CF9116
S1135F601F910F91FF90EF9008950F931F938FB798
S1135F70F894082F11278AE00E944C130FBF1F9139
S1135F800F910895FB01DC010D900020E9F71197B2
S1135F9001900D920020E1F708955058192EF7D082
S1135FA001D0DAC0BA176207730784079507B1F105
S1135FB088F40EF410940B2EBA2FA02D062E622F07
S1135FC0202D072E732F302D082E842F402D092EBF
S1135FD0952F502DFF275523B9F0591B49F0573EF3
S1135FE098F0469537952795A795F0405395C9F7AE
S1135FF076F0BA0F621F731F841F30F4879577956C
S11360006795B795F040939517FA0F2E0895BF1B27
S1136010BB27BA0B620B730B840BF6CFDEF6D4C02E
S1136020592F482F372F262F9FE380E8772766279D
S1136030AED001D091C0552359F0992369F09F57F0
S11360405F57951B33F442F4903811F4915805C00E
S11360509BC091589F3F09F4B7C0BB271124621716
S11360607307840730F4660F771F881FBB1F915096
S113607098F311D00F920FD00F920DD0A0E82617ED
S1136080370748071B0609F0A048BA2F602D7F91F7
S11360908F9100240895A0E80024621773078407F1
S11360A0B10528F0621B730B840BB1090A2A660F31
S11360B0771F881FBB1FA69581F7089597FB73D0A0
S11360C09F3738F0FEE9F91B982F872F762F6B2F17
S11360D005C077C09695879577956795F150D0F769
S11360E03EF490958095709561957F4F8F4F9F4FAB
S11360F00895E89403C097FB0EF4F3DFB62F672FDF
S1136100782F892F9EE9002427C00ED05EF004C0AA
S11361100BD026F001C008D019F020F48FEF0895B9
S113612080E0089581E0089597FB092E052600F884
S1136130689430D0E89407FC07C06217730784079B
S1136140950721F008F400940794989408959A957B
S1136150BB0F661F771F881F11249923A1F0882382
S1136160B2F79F3F59F0BB0F48F421F4002011F41B
S113617060FF04C06F5F7F4F8F4F9F4F881F9795BD
S1136180879597F908951DC09FEF80EC0895052E1B
S1136190092607FA440F551F5F3F79F0AA27A51770
S11361A008F051E04795880F991F9F3F31F0BB27B6
S11361B0B91708F091E0879508959F919F91112454
S11361C0E3CF66277727882799270895592F482FE3
S11361D0372F262FDCDF01D0BFCF992339F0552389
S11361E029F09F575F57950F13F4CAF1EDCF9158DB
S11361F09F3FE1F3A62F00241124BB2766275527D0
S1136200F8E0A69520F4020E131EB41F651F220F9A
S1136210331F441F551FFA95A1F7F8E0E72F77279E
S1136220F8E0E69520F4130EB41F651F7A1F330FB0
S1136230441F551FAA1FFA95A1F7F82F8827F69532
S113624020F4B40F651F7A1F8E1F440F551FAA1F19
S1136250EE1FFF23A1F788231AF4939539F494CF02
S1136260000C111CBB1F661F771F881F012808958F
S1136270629FD001739FF001829FE00DF11D649F26
S1136280E00DF11D929FF00D839FF00D749FF00DB2
S1136290659FF00D9927729FB00DE11DF91F639F53
S11362A0B00DE11DF91FBD01CF0111240895991B03
S11362B079E004C0991F961708F0961B881F7A95F9
S11362C0C9F780950895AA1BBB1B51E107C0AA1FFB
S11362D0BB1FA617B70710F0A61BB70B881F991F83
S11362E05A95A9F780959095BC01CD010895A1E236
S11362F01A2EAA1BBB1BFD010DC0AA1FBB1FEE1F3C
S1136300FF1FA217B307E407F50720F0A21BB30B86
S1136310E40BF50B661F771F881F991F1A9469F702
S113632060957095809590959B01AC01BD01CF015E
S10563300895CA
S113633201007DABBA83AAAA0120202020202025B7
S113634275203A2025750A0052636F756E742025F4
S1136352752053636F756E7420257520456E6572C2
S11363626779545820257520456E657267795258AD
S113637220257520456E6572677953502025750A6C
S1056382000015
S9030000FC
